:1030000039C0000052C0000050C000004EC0000097
:103010004CC000004AC0000048C0000046C000008C
:1030200044C0000042C0000040C00000B5C4000021
:103030003CC000003AC0000038C0000036C00000AC
:1030400034C0000032C0000030C000002EC00000BC
:103050002CC000002AC0000028C0000026C00000CC
:1030600024C0000022C0000020C000001EC00000DC
:103070001CC0000011241FBECFEFD2E0DEBFCDBFC9
:1030800011E0A0E0B1E0E6E6FDE302C005900D929C
:10309000A636B107D9F711E0A6E6B1E001C01D924E
:1030A000A438B107E1F762D35CC6AACF982F15C048
:1030B0008091F200882371F48091E8008B7F8093E7
:1030C000E80003C08EB3882351F08091E80082FFAE
:1030D000F9CF02C08091F1009150992349F70895EA
:1030E000209175013091740180917301909172016A
:1030F0008093670190936801C9018093690190935F
:103100006A0108951F93DF93CF9300D000D000D0C1
:10311000CDB7DEB780916D018823D9F08091700121
:10312000843049F480917101882339F480917201CF
:103130008F3F19F40EC0853061F08AE08093000162
:1031400083E080936C018091EB0080628093EB00C0
:10315000E3C080917001843009F458C0853030F4A8
:10316000813059F0833009F0D7C01DC0853009F493
:10317000A0C0863009F0D0C0C3C0109171011230D8
:1031800008F0CAC0ADDF112361F48091670190910E
:10319000680123E0FC0120935700E89507B600FC86
:1031A000FDCF85E008C080917101882311F0823045
:1031B00029F496DF89E080930001AEC0813009F0E8
:1031C000ABC020E030E040E050E0F90184918F3F57
:1031D00081F0CA01AA27BB2780936B013093680155
:1031E000209367018AE08093000185E080936C0161
:1031F00093C02F5F3F4F4F4F5F4F2030F0E33F07AB
:10320000F0E04F07F0E05F0701F786C080917101A1
:10321000833051F581E08093660180917601909131
:103220007701892B71F080917201813009F074C0AF
:10323000809175019091740190936F0180936E015C
:103240006BC080917201882361F42CE088E190E0EA
:103250000FB6F894A895809360000FBE209360008D
:103260005BC01092010158C0882309F055C08091BD
:1032700072018F3F09F050C0E0E0F0E093E085E09C
:1032800090935700E89507B600FCFDCF8093570058
:10329000E89507B600FCFDCFE058FF4F20E3E03093
:1032A000F20771F781E180935700E89510926D0164
:1032B00033C0DE011196E5E0F1E083E001900D926C
:1032C0008150E1F7DE011496E2E0F1E083E0019045
:1032D0000D928150E1F790917201809171018823E4
:1032E00029F4FE01E90FF11D818107C08130A1F4AD
:1032F000FE01BC97E90FF11D8081809378010CC01D
:1033000080917101833041F480917201882321F40E
:103310008091730180936B0126960FB6F894DEBFFF
:103320000FBECDBFCF91DF911F9108952F923F9295
:103330004F925F927F928F929F92AF92BF92CF9265
:10334000DF92EF92FF920F931F93DF93CF9300D002
:10335000CDB7DEB700918201109183011093770100
:103360000093760180917C018F77813209F0EAC168
:1033700080917D01833009F4AFC1843030F4813015
:1033800071F0823009F0DEC112C1853009F4C2C18A
:10339000853008F4B7C1863009F0D4C1CAC1809124
:1033A000E800877F8093E80080916601882319F008
:1033B000A9DE109266010115110529F42BC08EB308
:1033C000882309F4BFC18091E80082FFF8CF809183
:1033D000F1008093700198012150304030937701C3
:1033E00020937601E1E7F1E00CC08091F100819338
:1033F0002150304061E0E637F60719F4318320832D
:1034000008C08091F200882381F7309377012093E0
:10341000760178DE80910001853009F0C4C080918A
:10342000760190917701892B21F482E0809300014D
:10343000BAC08AE13BDEE0906701F09068018E2D12
:103440008F7134DE8090690190906A010894811C2C
:10345000911C84010E191F0908948108910880911C
:103460007101882309F09AC0C801969587959A83BF
:103470008983C701A0916B01B0E09C01AD0162E0BE
:10348000E62EF12C012D112DE20EF31E041F151F47
:1034900059016A0190E077247394B5E0A3E04CC031
:1034A0008091F200882371F48091E8008B7F8093F3
:1034B000E80004C08EB3882309F444C18091E80079
:1034C00082FFF8CFE981FA813197FA83E98380910D
:1034D000F100682F8091F100782FF5010B017092B7
:1034E0005700E89511249F5F903421F029803A809D
:1034F0002328A9F4F901B0935700E89507B600FC1A
:10350000FDCF29803A80232851F0F701A09357007E
:10351000E89507B600FCFDCFA801970190E042E0D6
:10352000242E312C412C512CE20CF31C041D151DB2
:10353000A20CB31CC41CD51C49805A80452809F034
:10354000AFCF909268018092670181E1809357002C
:10355000E89527C08091F200882371F48091E800FB
:103560008B7F8093E80004C08EB3882309F4EAC0FF
:103570008091E80082FFF8CF6091F10080916701AF
:1035800090916801E0D38091670190916801019664
:103590009093680180936701015010400115110557
:1035A000C9F680E183DD8091E8008B7FBFC0809108
:1035B000E800877F8093E80004C08EB3882309F475
:1035C000C1C08091E80080FFF8CF80910001893070
:1035D00091F08A3069F480917101813049F48091D1
:1035E0006701909168018093F1009093F1009BC076
:1035F0008091780196C06091690170916A01209173
:103600006701309168016F5F7F4F7B01E21AF30A17
:103610006150704080917101882389F5870116956A
:103620000795C901A0916B01B0E09C01AD011FC0DD
:103630008091F200803271F48091E8008E7F809357
:10364000E80004C08EB3882309F47CC08091E800B0
:1036500080FFF8CFF901859194918093F1009093C8
:10366000F100015010402E5F3F4F4F4F5F4F01154B
:103670001105F1F6709368016093670129C08230EB
:1036800039F523C08091F200803271F48091E80016
:103690008E7F8093E80004C08EB3882309F452C063
:1036A0008091E80080FFF8CF0091670110916801D8
:1036B000C80141D38093F1000F5F1F4F1093680141
:1036C000009367010894E108F108E114F104D1F6D0
:1036D00082E08093000127C08091E800877F80937B
:1036E000E80080916C018093F1001092F10010923B
:1036F000F1001092F100809100018093F10010928E
:10370000F10011C08091E800877F8093E80010925B
:103710006C0117C08091E800877F8093E80080915A
:1037200000018093F1008091E8008E7F8093E80093
:1037300008C08091E800877F8093E80082E0809352
:103740000001B2D00F900F90CF91DF911F910F9198
:10375000FF90EF90DF90CF90BF90AF909F908F90B1
:103760007F905F904F903F902F90089584B7809303
:10377000840184B7877F84BF88E10FB6F894809373
:103780006000109260000FBE90E880E00FB6F894E1
:1037900090936100809361000FBE8091630081600F
:1037A000809363008FE785B984E088B981E98BB99C
:1037B00045983D9A44983C9A27982F9A3E98469A65
:1037C000E0EEFEE23197F1F75E98569A5998519AD9
:1037D0008091640084608093640090BF449A83B1B8
:1037E00096B19095907487FD04C0992331F481E0DF
:1037F0001AC0992309F583E016C081E085BF82E0F5
:1038000085BFBBD0789401C08DD2809101018823FF
:10381000D9F7809166018823B9F765D0F89481E0E3
:1038200085BF15BE80E08ABD809184018BBDE0918B
:103830006E01F0916F01099582E0F5CFFA019230A7
:1038400071F0933089F0913029F488E091E022E121
:1038500030E015C080E090E020E030E010C08AE168
:1038600091E02BE130E00BC0882329F485E391E05F
:1038700024E030E004C089E391E02AE230E0918363
:103880008083C90108958091EB0081608093EB00F3
:103890001092ED006093EC004093ED008091EE00FB
:1038A000881F8827881F089580917C0188238CF4C5
:1038B00003C08EB38823B1F08091E80082FFF9CF76
:1038C0008091E8008B7F8093E80008958EB3882371
:1038D00049F08091E80080FFF9CF8091E8008E7F69
:1038E0008093E800089552D054D0E0EEF0E080815B
:1038F00081608083E8EDF0E080818F77808319BC60
:10390000E3E6F0E080818160808310927B0108957E
:103910003DD03FD08091D800982F9F779093D800CA
:1039200080688093D8008091D8008F7D8093D800E4
:1039300019BC89B5826089BD09B400FEFDCF1EBAED
:1039400010927A011092790180E060E042E29BDF00
:103950008091E1008E7F8093E1008091E2008160A0
:103960008093E2008091E20088608093E200809181
:10397000E0008E7F8093E0000895E3E6F0E0808130
:103980008160808381E080937B01C2CF1092E2004E
:1039900008951092E10008951F920F920FB60F92B2
:1039A00011242F933F934F935F936F937F938F9344
:1039B0009F93AF93BF93EF93FF938091E10080FFBC
:1039C00016C08091E20080FF12C08091E2008E7FDD
:1039D0008093E2008091E20080618093E200809118
:1039E000D80080628093D80019BC1EBA3ED1809165
:1039F000E10084FF2CC08091E20084FF28C019BC44
:103A000089B5826089BD09B400FEFDCF8091D800E0
:103A10008F7D8093D8008091E1008F7E8093E100BC
:103A20008091E2008F7E8093E2008091E2008160CD
:103A30008093E20080917A01882331F48091E30041
:103A400087FD02C081E001C084E08EBB0ED1809171
:103A5000E10083FF21C08091E20083FF1DC08091BF
:103A6000E100877F8093E10082E08EBB10927A01B3
:103A70008091E1008E7F8093E1008091E2008E7F53
:103A80008093E2008091E20080618093E20080E018
:103A900060E042E2F8DEE9D0FF91EF91BF91AF9193
:103AA0009F918F917F916F915F914F913F912F9156
:103AB0000F900FBE0F901F9018950F931F93DF93D9
:103AC000CF9300D0CDB7DEB78091F10080937C0119
:103AD0008091F10080937D018091F1009091F1003F
:103AE000EEE7F1E080937E0190937F018091F100F9
:103AF0009091F1008093800193838091F1009091E7
:103B0000F10080938201958311DC8091E80083FFAE
:103B100097C090917C0180917D01863009F443C06B
:103B2000873030F4882359F0853009F089C016C0F9
:103B3000883009F458C0893009F082C066C09038D6
:103B400009F07EC0809179019091E800977F909371
:103B5000E8008093F1001092F10050C0992309F021
:103B60006FC010917E011F770FB7F8948091E80025
:103B7000877F8093E80098DE8091E80080FFFCCF8B
:103B80008091E3008078812B8093E3008091E300B3
:103B900080688093E300112311F482E001C083E088
:103BA0008EBB0FBF4DC09058923008F049C0809135
:103BB0007E0190917F0160918001AE014F5F5F4F68
:103BC0003DDEBC01009709F43BC08091E800877F8F
:103BD0008093E80089819A8149D08091E8008B7FA9
:103BE0008093E8002DC0903859F58091E800877FD8
:103BF0008093E80080917A018093F1008091E80041
:103C00008E7F8093E80050DE1BC09923C9F4909109
:103C10007E019230A8F48091E800877F8093E800CD
:103C200090937A0141DE80917A01882331F480916A
:103C3000E30087FD02C081E001C084E08EBB15D0A7
:103C40008091E80083FF0AC08091EB00806280933E
:103C5000EB008091E800877F8093E8000F900F9041
:103C6000CF91DF911F910F91089508959C0140918C
:103C70008201509183014617570718F4F90190E02B
:103C80003CC06115710511F0AB01F8CF8091E800DF
:103C90008E7F8093E80040E050E0F0CF8EB3882321
:103CA000E9F18530E9F18091E80083FF02C081E00D
:103CB00008958091E80082FD2BC08091E80080FF8C
:103CC0001CC08091F200282F30E007C081918093C2
:103CD000F100415050402F5F3F4F4115510519F001
:103CE0002032310598F390E02032310509F491E05B
:103CF0008091E8008E7F8093E8004115510571F6B0
:103D0000992361F605C08EB3882341F0853041F0D8
:103D10008091E80082FFF7CF80E0089582E0089567
:103D200083E008958EB3882329F08091E80083FF13
:103D300001C0C3CE0895F999FECF92BD81BDF89A16
:103D4000992780B50895262FF999FECF1FBA92BD05
:103D500081BD20BD0FB6F894FA9AF99A0FBE01966C
:063D60000895F894FFCF66
:103D660002011E948220DCFB1201100100000020DB
:103D7600EB03FA2F00000001000109021B000101FC
:103D860000C0640904000000FE01020009210300CE
:103D960000000C0001040309042A034D0054002D01
:103DA6000058003100200044004600550020004223
:103DB600006F006F0074006C006F006100640065A6
:063DC60000720000000085
:0400000300003000C9
:00000001FF
